:020000040000FA
:020000000528D1
:0800080010288316003085006A
:10001000FF308600831286019301640011200D28B1
:100020000D288520930106181314861893140619B9
:10003000131586199315061A1316861A9316061B9E
:100040001317861B9317851405141430920085200E
:10005000920B2728051085208520852085200514F2
:100060008520131C352885208520051085208520B6
:100070008520852005148520931C40288520852017
:100080000510852085208520852005148520131DD9
:100090004B288520852005108520852085208520FA
:1000A00005148520931D5628852085200510852060
:1000B00085208520852005148520131E6128852034
:1000C0008520051085208520852085200514852024
:1000D000931E6C288520852005108520852085208D
:1000E000852005148520131F77288520852005107D
:1000F000852085208520852005148520931F822852
:10010000852085200510851008000A3091001430E4
:0E0110009000900B8928910B8728640008004E
:00000001FF
